:10000000B86D0010A5010000A9010000AB010000BF
:10001000AD010000AF010000B10100004288FFEF18
:10002000000000000000000000000000B30100001C
:10003000B501000000000000B7010000B901000098
:10004000BB010000BB010000BB010000BB010000C0
:10005000BB010000BB010000BB010000BB010000B0
:10006000BB010000BB010000BB010000BB010000A0
:10007000BB010000BB010000BB010000BB01000090
:10008000BB010000BB010000BB010000BB01000080
:10009000BB010000BB010000BB010000BB01000070
:1000A00043260000BB010000BB010000BB010000B3
:1000B000BB010000BB010000BB010000BB01000050
:1000C000BB010000BB010000BB01000000F002F812
:1000D00000F03EF80AA090E8000C82448344AAF1A4
:1000E0000107DA4501D100F033F8AFF2090EBAE8A2
:1000F0000F0013F0010F18BFFB1A43F0010318475C
:100100006454000084540000103A24BF78C878C1B9
:10011000FAD8520724BF30C830C144BF04680C600D
:10012000704700000023002400250026103A28BF55
:1001300078C1FBD8520728BF30C148BF0B60704759
:100140001FB59DE8030004F0A6FD1FBD10B510BD4E
:1001500004F011FE1146FFF7F3FF00F01EFB04F060
:100160002FFE03B4FFF7F2FF03BC04F05FFE0000B4
:10017000D0F800D0D0F804F070B50023084D0AE0A4
:10018000CE5C04885B1C86EA14269BB235F81660A8
:1001900086EA04240480521E92B2F1D270BD00009F
:1001A000784F000008480047FEE7FEE7FEE7FEE75D
:1001B000FEE7FEE7FEE7FEE7FEE7FEE70348044949
:1001C000044A054B70470000CD000000B81D001028
:1001D000B86D0010B85D0010B85D0010064802212F
:1001E00041600021016741610B22C260C1630121AE
:1001F0004160002070470000008000402C48002132
:100200000167C1600222426181613022C2632948D4
:1002100082682948C0E900210846704770B541F25C
:100220008832904215D8642800D290B942F21072F8
:1002300091420ED805290CD31E4CA2681E4B1D6896
:10024000521B5D6805EB4506C6EBC515B2EBC50F45
:1002500001D2002070BD164A0225556038B1174EF4
:10026000B6FBF0F040109061556001205060A0682E
:10027000C3E90001EDE770B50F4C00250E4665603F
:10028000FFF7CCFF0B4A06EB46012068C1EBC61115
:1002900093681B1AB3EBC10FFAD3054802214160E2
:1002A000C16B01F0FE01C1630020656070BD0000FC
:1002B0000000094000800040DC000010001BB70077
:1002C000EFF3108010F0010F72B64FF080404FF046
:1002D000000202704FF0AA0303724FF0550404723B
:1002E00002614FF0FF0242604FF00302027003729E
:1002F000047200D162B6FEE770477047FFFFFFFF50
:1003000070B5284C607820B30026274D012810D006
:1003100002280DD1A8686168401A2449884215D383
:100320002348406B400011D5012002F064F866704C
:1003300070BDA8686168401A1E498842F8D3002041
:1003400002F059F8A86860600220607026700C20E6
:1003500005E020780028EBD1012020700D20BDE8B9
:10036000704001F0E7B8002802D10E490120487022
:10037000704710B501F05CFD0A490020487010BDBF
:1003800008480121417008498968416070477047F9
:100390007047022803D0032803D100F0AEBD00F05F
:1003A000C9BD70470801001000800040A086010010
:1003B00000C0092040420F0010B591FBF2F491FB00
:1003C000F2F302FB1411C0E9003110BD7047704711
:1003D0007047000000487047601D00100021016058
:1003E000C0E90110704710207047000000487047B6
:1003F000581D001010B504F0F1FCBDE8104004F0E9
:10040000E8BC70474D0B0000FD4910B5486D000574
:100410000CD4FC4A906843F698239468241A9C42B2
:10042000FBD3486D000501D4012010BD052001F06B
:1004300081F8002010BD70B5F24CA668042001F0D0
:1004400079F8F14D03E000BFFFF7DEFF48B1A06887
:10045000801BA842F8D308E0FFF7D6FF08B10120BF
:1004600070BDA068801BA842F6D3002070BD2DE9A6
:10047000F041092001F05EF8E44800264FF47A7755
:100480000670C8213846FFF7F6FEDE4CA06842F23F
:100490001075A168091AA942FBD3C8213846FFF795
:1004A000EAFEA068A168091AA942FBD3C821384610
:1004B000FFF7E1FED648022186708171C670BDE863
:1004C000F0818AB046208DF814004FF000098DF8B5
:1004D000179036208DF81500CE4A37208DF816007B
:1004E0001068CA464FF6FF031840CB4B40F48070AB
:1004F00018431060C948CB49CD4DC0F80090C8489A
:100500000068A0F56C50FF380860C74900F5E0505E
:100510000860C649400A0860F8202870FF2068700B
:10052000A870FFF76BFEBA4CC24A002094F9051080
:1005300052F821102B1803F580530A5C401C83F8F5
:1005400000286028F6D34FF4E175294640F249109F
:10055000FFF791FE294640F29F10FFF78CFE4FF403
:10056000005BDFF8D4825D46207808B1FFF7C8FE53
:10057000A07928B1012818D02078002879D0FCE093
:100580000A2000F0D7FF00F00FFE10B1FFF76FFF59
:10059000EAE70120A0715D4684F803A0062000F080
:1005A000C9FF0A2000F0C6FFDEE719222946A2484B
:1005B00000F0BAFD98F8180000287CD098F80000E8
:1005C000062873D2DFE800F072030B46464940F27A
:1005D000044000880390D8F80410814266D098F84F
:1005E00009104FF00109404601295FD1D0F80A10E7
:1005F00019B992498969C0F80A100026804617E0A7
:10060000072000F097FFD7F80E00B846871B402F51
:1006100000D94027A9193A468948193100F084FDCC
:10062000D8F80A003A463044854900F0F1FE3E44CD
:10063000D8F80E004746B042E2D83978012935D1C2
:100640004FF0E0220906C2F88011D7F80A0000F046
:100650000DFF2BE04FF001092BE098F809104FF047
:100660000109032925D16E49764A00260B681360DB
:1006700017E07BE0072000F05DFFD7F80E00871B36
:10068000402F00D94027A9193A466D48193100F08A
:100690004BFD63483A4600688119694800F033FD14
:1006A0003E44D8F80E004746B042E3D898F8180008
:1006B00008B1464600E01CE098F80800C00613D5D3
:1006C0006049012203A8C1F800B005F11801CDF876
:1006D0000CA000F009FD307820B1C8214FF47A70E9
:1006E000FFF7C9FD307E20B1307A800701D5FFF7D2
:1006F000E7FDD8F80E001B3505444F4800F048FDD3
:1007000030B302204149A0715D4681F800A00B2062
:1007100000F010FFB9F1000F1AD03A484FF000096D
:10072000816842F2107283685B1A9342FBD34FF4E4
:100730002F714FF47A70FFF79EFD3148406D4005F0
:1007400002D50020099001E0099808B9FFF7B8FD2B
:10075000E078401CC0B2E0700C2802D30120A070E9
:1007600014E7A07800283FF413AF0FE701202070B2
:1007700001F080FE012001F03EFE244800780028B0
:10078000F1D0002105A800F021FC0028EBD084F86E
:1007900006A05D4684F803A0E6E61D4C0026FF2077
:1007A0002660A680A671607100F064FF01F010F869
:1007B000FFF714FD00F084FE002000F0BBFE01F006
:1007C000C1FFFFF721FEF8B3042000F0B3FE0C4F89
:1007D000786D0C4D00053AD4FFF72DFEA0B3FFF75E
:1007E0002AFE88B3FFF727FE70B3042000F0A2FEB4
:1007F000A86805497A6D120529D4AA68121A24E05E
:1008000000C009200080004080841E0068000010A5
:10081000BC0000100CED00E00000FA05AC00001078
:10082000B80000109C000010940000109800001008
:1008300035010010600000101C010010B8520000CB
:10084000AD1B0010B000001009E08A42D2D3A868A6
:1008500042F21071AA68121A8A42FBD3667100F044
:1008600035FC00F0A1FC80B100F007FE68B1022069
:1008700000F060FE94F90500401C03D10C4880692B
:1008800000F0F4FD0120607004E0022000F052FE50
:1008900066706671FFF7B8FD40B14021054804F06D
:1008A000C2F94022D101034800F02DFCFFF709FEF8
:1008B000B8520000AD1B00102DE9F047FE4A00239E
:1008C0004FF40077156A4FF4FF79C5F30724DFF87A
:1008D000ECA34FF4E05CDFF8E883FA4E25E0B84281
:1008E00016D213280CD014280CD048450CD0A0F5F3
:1008F0008072FF3A0AD03E2813D81AF8002011E07F
:10090000EAB20FE022460DE055220BE0AA2209E0F0
:10091000604506D208EB0002A2F5805292F8002E44
:1009200000E00022F254401C5B1C8B42D7D3BDE890
:10093000F08770B5E04D2C6B402C00D94024E86A5C
:10094000E96902198A4202D90C1A04216970214608
:10095000FFF7B2FF2246DB49822001F048FEE86A39
:100960002044E862286B011BD74829638268A2EB08
:100970000402826005D06978022901D00021017348
:1009800070BD03216970F9E7CF4910B5CF48086001
:100990000D22822001F02BFEC7490520487010BDB2
:1009A00070B50D46CA49496D490521D4B0F5007F9F
:1009B0001ED3C849C04CB0F5E05F1AD28A68A3695B
:1009C000D21AC54B9A4204D38968A16100216160A3
:1009D0006161BD4900235F39B94A07E0C418144476
:1009E000CE5CA4F580545B1C84F8006EAB42F5D35A
:1009F00070BD626922B98A68A2618A686261A0607A
:100A0000B64A5279002AF3D18A686369D21AB44B84
:100A10009A421CD2B34B01221A708A68A26189687B
:100A20006161A168401A6168884203D9616A88429D
:100A300000D26060062000F07DFD61682A46BDE8B6
:100A40007040A14801F500515F3800F05CBBBDE883
:100A500070400C2000F06EBD10B5974CA178E06A94
:100A60004218E1698A4206D9081AA0700520607010
:100A7000022001F077FDA178E06AFFF791FFA178ED
:100A8000E06A0844E062206B421A8F482263836860
:100A9000A3EB0101816002D06178052904D1002116
:100AA0000173BDE810406FE710BD2DE9F041824CA5
:100AB000A178E06A4218E1698A4206D9081AA07052
:100AC00005206070022001F04DFD7F4D0021A078CF
:100AD0007C4B5F3DE26A08E056186F5C9E5DBE424B
:100AE00002D00021A16202E0491C8142F4D3111816
:100AF000E162216B0A1A744922638B68A3EB000040
:100B0000886002D06078052808D1A06A20B1002052
:100B10000873BDE8F04137E70120F9E7BDE8F0814F
:100B2000694810B51F38D0F81110027D09BA21F0BC
:100B3000FF011143604A4902D162C18A49BA4902A0
:100B40001163806888420CD0822001F00BFD0220E6
:100B500001F008FD5C4902200873FFF715FF002033
:100B600010BD012010BD70B55748574D1F380224E5
:100B7000816829B1007B000607D4022001F0F2FC55
:100B80002C73FFF701FF002070BD012070BD10B570
:100B90004D48494C1F388068A178884200D2A07027
:100BA0004949A2785F39822001F021FD032060705D
:100BB0004548A2788168891A81600021017310BDBF
:100BC000414810B51F38816839B1007B000601D556
:100BD000822000E0022001F0C5FC3B4900200873A0
:100BE000BDE81040D0E610B5FFF7BDFF00281FD0CC
:100BF000354870215F3802220170002141708270F7
:100C0000C1700171417181710A22C2710172417218
:100C10008172C17230220273012242738173C173E7
:100C200001744174244912208870BDE81040AEE779
:100C300010BD1CB5FFF797FF00286AD02A480A228A
:100C400006210388684600F025FA1F4800225F3815
:100C500080230270437082700121C17020210171D4
:100C600043718271C27141220272542242724F2238
:100C700082724C22C272017341738173C173462226
:100C8000027450234374722383746923C3746E23E4
:100C90000375742343758175C2756C2202766122D7
:100CA0004276732282766822C27601774177817715
:100CB000C1779DF8011019E078000010785200000B
:100CC00035010010AD1B0010941B0010555342530A
:100CD00000C0092000800040A0860100BC00001078
:100CE00020A10700680000100404000080F8201014
:100CF0009DF8021080F821109DF8031080F8221052
:100D00009DF8041080F82310DE4924208870FFF736
:100D10003EFF1CBD10B5FFF726FF00280CD0DA48B7
:100D200003210170002141708170C170D5490420F8
:100D30008870BDE810402AE710BD10B5FFF713FF1B
:100D4000002810D0D0480021062201704270817026
:100D5000C170017141718171C171CA4908208870E7
:100D6000BDE8104013E710BD10B5FFF7FCFE0028EA
:100D700015D0C44AC448116A491E0B0E03700B0CEF
:100D800043700B0A8370C17000210171417102230D
:100D90008371C17108209070BDE81040F7E610BD66
:100DA00010B5FFF7E0FE002819D0B7480021B54B79
:100DB0000170417081700822C2701A6A140E0471A9
:100DC000140C4471140A8471C271022202724172BD
:100DD0008272C1720C209870BDE81040D7E610BD39
:100DE0002DE9F041A74DA84C0021A8784034A64A2F
:100DF00002E0535C6354491C03468142F9D31F2B24
:100E000072D12068A14988426ED19F4E60685F36DA
:100E10004FF001087060A068B060607B18B9A07BDB
:100E200008B1102802D986F80C8059E0E07B1E2812
:100E3000F9D00FDC12282ED005DC48B30328F2D1FC
:100E4000BDE8F041CFE61528EDD01A28EBD1BDE87A
:100E5000F0415FE702272A2828D010DC23281DD084
:100E600025281ED02828DED1FFF75AFE002826D0DC
:100E7000207B000618D56F70BDE8F04159E52F289A
:100E80001ED05528CFD05A28CDD1BDE8F04154E727
:100E9000BDE8F04194E6BDE8F041CAE6BDE8F041A6
:100EA0007EE7BDE8F0415FE7022016E0FFF738FE7D
:100EB000002804D0207B00060ED485F801802DE6A2
:100EC000FFF72EFE0028FAD0207B000604D485F818
:100ED0000180C5F8288021E6822001F043FB3773AA
:100EE000BDE8F04150E5FFE7822001F03BFB022026
:100EF00001F038FB0620687010E6624810B54178B2
:100F0000022908D003290ED004290FD0052901D1C8
:100F10000021417010BD5C484030C07B2828F9D1C9
:100F2000BDE8104005E5BDE810402DE5822001F048
:100F300019FBF8E710B55449022001F027FB51498D
:100F40008870487858B101280CD0022001F00AFBC3
:100F50004D4902205F310873BDE8104014E5BDE83B
:100F600010403DE748484030C07B2A2804D02F2855
:100F700005D1BDE8104098E5BDE810406CE510BD16
:100F8000FFB50246002002EB420501464FF44056F1
:100F90006C4603AA6B1844F82130B34202DD0020EE
:100FA00004B0F0BD3A4F07EB6307DB073F785754B7
:100FB00001D03B095354535C8F0003F00F0353548B
:100FC000BB40491C18440329E4DBE9E7F0B50646B9
:100FD0000020034602462E4C4FF4007700E05B1CD5
:100FE000F55C45B102EB030CA4440CF5805C9CF865
:100FF00000C8AC45F3D0032B3FD302F5C0502044CA
:10100000037F457FC67F03EB0523857F2D0405EB1A
:1010100006652B4451EA03052BD021B919494968CB
:1010200040318B4225D8184B00216C33551825448C
:1010300005F5805595F800585D54491C0C29F5D3E9
:10104000817EC27E01EB0221027D407D120402EB13
:1010500000600C182046FFF793FF40F6F57501E09D
:10106000FFF78EFFC11EA942FAD3A0F57061FF39C8
:1010700001D00020F0BD2046F0BD2032BA42AFD3EF
:10108000F0BD000078000010351B0010555342439E
:1010900035010010FFB5ACA60446E1CE8DE8E100B5
:1010A000022902DA002004B0F0BD6018002100F827
:1010B000011D6946B3FBF2F502FB1535B3FBF2F3F4
:1010C0004D5D00F8015DA042F4D8ECE710B503F0E7
:1010D0001FFC03F009FCA0494FF40052C1E90020B5
:1010E000A0F5F420886010BD70B5034608468D1841
:1010F0009949002449688D4200D9881A194603F09D
:1011000055FC204670BDF8B51446934E0A460B199F
:10111000716800258B4200D90A1B03460094306891
:1011200003F06FFC2846F8BD10B50B4601460024BD
:10113000184603F010FC204610BD2DE9FC4107467F
:10114000002090460E46ADF8000004460EE0351B28
:10115000402D00D9402539192A468048FFF7E4FF81
:10116000AAB27E496846FFF707F82C44B442EED392
:101170003919424601A8FFF7D7FFBDF80000BDF8B6
:101180000410884202D10120BDE8FC810020FBE769
:101190000021425C12B9491C1829FAD3182901D040
:1011A00000207047012070472DE9F0416A4C00276C
:1011B0000C3488B0A770E770DFF8A4814FF40056B4
:1011C000277101251922314601A8FFF7ADFF022240
:1011D00016213046FFF7B1FF00287DD0DDF8121050
:1011E000022206F11900FFF7A8FF002874D09DF82D
:1011F0000400062829D2DFE800F029030329291C6E
:10120000D8F87410DDF80E30491C8B421DD2D8F886
:101210007420DDF80E30D21ADDF81230521C9A42DA
:1012200013D3DDF80E20DDF812301A448A420CD8B0
:101230000CE0DDF81210B1F5F42F00D9A570DDF83F
:101240001610C1F30B41112900D0A570012803D05D
:10125000022801D0052839D1022206F21D41684634
:101260000097FFF761FF0099029889B2884200D089
:10127000A570012206F2254168460097FFF754FF4A
:101280000099BDF80500C9B2884200D0A5709DF84C
:10129000040002281AD1042206F249416846009748
:1012A000FFF742FFDDF816000099884200D0A570D4
:1012B000012206F24D4168460097FFF735FF00987E
:1012C0009DF80710C0B2814200D0A5709DF81C00A7
:1012D000401EFE2802D200E01EE0A570BDF8050009
:1012E000A0F57F41FF3901D0432802D19DF80700C6
:1012F00020B901A8FFF74CFF00B9A570DDF8120076
:101300001B36064401A8FFF743FF30B1E07880B1F7
:10131000217988420DD012E0A5709DF81C0010B90B
:101320002079401C2071E078401CC0B2E0700C288D
:1013300001D3A57003E0A07800283FF443AFA07864
:1013400008B0BDE8F0810000303132333435363733
:101350003839414243444546B0000010AD1B0010EF
:10136000305300004F4A104710B572B633244E4B2D
:1013700010C307C34D484FF47A710068B0FBF1F019
:101380001860191D4848FFF7EDFF62B610BD464AC8
:1013900032231360C2E9010144484FF47A710068B6
:1013A000B0FBF1F0D06002F114011046DAE73E4ADA
:1013B00034231360C2E901013C484FF47A7100689C
:1013C000B0FBF1F0D06002F114011046CAE710B58D
:1013D00072B60624364900BF51F82420824212D941
:1013E0003349783951F82410814207D12146084603
:1013F000FFF7CDFF21460846FFF7D9FF21460846F3
:10140000FFF7C5FF02E0641C1D2CE5D962B610BDD4
:101410002DE9F041274C236803B92060224D0020BC
:101420002835636803E00F5C1E18401CAF559042DE
:10143000F9D398184FF480766060B04213D12068D9
:10144000FFF7C5FF184D1435286800B1FEE71649AF
:10145000324628312068FFF787FF286800B1FEE791
:101460000020606020600020BDE8F08172B6124963
:10147000124A01401160FEF77BBE46F20440002193
:101480000088A0F51942993A0AD04FF4C0404FF4B1
:10149000002208C890421944FBD309B100207047CC
:1014A00001207047F11FFF1FF01B0010D800001033
:1014B00030530000C400001080FFFF1F08ED00E063
:1014C000002070476949C20702D04FF480028A6148
:1014D000800702D54FF400108861002070476349EF
:1014E000C20702D04FF48002CA61800702D54FF4D0
:1014F0000010C86100207047014600205B4ACB07FE
:1015000003D053695B0200D50120890704D55169D6
:10151000890201D540F00200704710B50446FFF77C
:10152000EBFF0346FFF7DBFF24EA0300FFF7CAFFE8
:10153000002010BD70B54E4B50B1596804240325EE
:101540000226052907D2DFE801F0072B4A718E0039
:1015500000205860986070BD042807D0052809D085
:10156000012402287AD0012808D00FE00320FFF7D9
:10157000B6FF46E0BDE870400120B0E70320FFF76A
:10158000AEFF0BE0FFF79EFF5C6070BD0E28FCD144
:101590000320FFF7A4FF0220FFF794FF0120F1E7EB
:1015A00006280AD0032810D00A2813D0092811D001
:1015B0000D280FD00C28D9D070BD0320FFF78FFF66
:1015C0000220FFF77FFF5E6070BD0320FFF787FFFB
:1015D000012027E00320FFF782FF022012E0062807
:1015E00013D00A281AD00928C8D00C28BED00D283C
:1015F000F0D00F28E8D10320FFF771FF0220FFF79A
:1016000061FF0120BDE870405CE7986810F01F0F93
:1016100000F101009860D7D102201BE00320FFF702
:101620005EFF0220FFF74EFF5D6070BD072806D009
:101630000A289BD00B2811D009289FD070BD02200A
:10164000FFF74DFF986810F03F0F00F10100986020
:10165000F4D10120BDE870405FE7FFE70320FFF70A
:101660003EFF02208EE70628A7D08FE700C00920A2
:10167000CC0000104F4810B52021C0F8A01100BFC9
:10168000D0F8A0114906FBD50521C0F804114FF090
:101690004472C0F8A8214FF48062C0F8AC21012246
:1016A000C0F80C210B23C0F88430C0F88020AA2297
:1016B000C0F88C205523C0F88C3000BFD0F888408B
:1016C0006401FBD50324C0F88040C0F88C20C0F82A
:1016D0008C30C0F808113849C0F8C4100021C0F897
:1016E000C811D0F888106FEA11618A073349D0F821
:1016F0000C2102F0030207D07AB3012A44D0022A57
:1017000047D0032A4ED13AE02AB1012A13D0022A47
:1017100024D0032A46D1D0F88820D0F80431C2F36F
:101720000742DBB2521C5B1C5A43D0F88830244C71
:10173000C3F30E030EE0D0F88820D0F80431C2F3D2
:101740000742DBB2521C5B1C5A43D0F888301D4C58
:10175000C3F30E035B1C634321E010E0D0F8882044
:10176000D0F80431C2F30742DBB2521C5B1C5A436F
:10177000D0F888304FF47A44C3F30E03EAE7D0F888
:101780000421114BD2B209E0D0F804210F4BD2B2A0
:1017900004E0D0F804214FF4FA43D2B2521CB3FB58
:1017A000F2F20A60016821F4704141F400510160D5
:1017B00010BD000000C00F40DC966883D800001008
:1017C00000127A0000366E0100093D00001BB700D0
:1017D000F0B5FF4800218162016821F440310160C9
:1017E000016C21F4403141F400310164F949831561
:1017F000CB610A6842F480720A60026822F44052A7
:101800000260026C22F4405242F400520264402210
:10181000CA610C6844F040040C60046824F440641D
:101820000460046C24F4406444F4006404642024E0
:10183000CC610C6844F020040C60046824F440740B
:101840000460046C24F4407444F4007404641024B0
:10185000CC610D6845F010050D60C56825F00C05DC
:10186000C560C56C25F00C0545F00805C564D502BA
:10187000CD630E6A46F400360E62066926F44056C1
:101880000661066D26F4405646F4005606658A65E4
:101890000A6C42F040020A64026922F00302521C00
:1018A0000261026D42F003020265026922F00C023D
:1018B000121D0261026D42F00C020265026922F003
:1018C000300242F010020261026D42F03002026505
:1018D000026922F0C00242F040020261026D42F051
:1018E000C0020265026922F4407242F48072026111
:1018F000026D42F440720265026922F4406242F4D1
:1019000080620261026D42F440620265026822F464
:10191000404242F400420260026C22F440420264FF
:10192000026822F4402242F400220260026C22F497
:1019300040220264426822F00C024260426C22F0B3
:101940000C024264CD610A6822F400320A604268E7
:1019500022F030024260426C22F0300242F020025B
:1019600042649D02CD610A6822F480220A60C26846
:1019700042F44022C260C26C22F4402242F40022AF
:10198000C264C26842F04042C260C26C22F040426F
:1019900042F00042C264026822F0300242F01002BB
:1019A0000260026C22F0300242F0200202640268FF
:1019B00022F0C00242F040020260026C22F0C0023B
:1019C0000264026922F040620261026D22F040620C
:1019D00042F0006202655A01CA650A6C42F4005284
:1019E0000A64026822F0404242F080420260026CC7
:1019F00022F0404242F000420264426822F00302B8
:101A0000521C4260426C22F003024264026922F4DA
:101A1000403242F400320261026D22F4403242F45C
:101A200000320265026922F4402242F4002202617F
:101A3000026D22F440220265026822F00302921C29
:101A40000260026C22F00302921C0264026822F01F
:101A50000C0242F008020260026C22F00C020264E6
:101A6000C26842F44032C260C26C22F4403242F496
:101A70000032C264C26842F44042C260C26C22F4C6
:101A8000404242F40042C264C26842F44072C26002
:101A9000C26C22F4407242F40072C264C26822F442
:101AA0004052C260C26C22F44052C2649E038E63F4
:101AB0000A6A42F480020A62C26822F44062C2608A
:101AC000C26C22F44062C2645A038A630F6A47F40C
:101AD00000170F62C76827F44017C760C76C27F468
:101AE0004017C76457018F63D1F820C04CF0806C59
:101AF000C1F820C0D0F80CC02CF0300CC0F80CC0DD
:101B0000D0F84CC02CF0300CC0F84CC08D630D6A7E
:101B100045F480250D62456825F0407545F08075D7
:101B20004560456C25F040754564456825F44005E1
:101B300045F480054560456C25F4400545644568DD
:101B400045F440754560456C25F44075456445682D
:101B500045F0C0054560456C25F0C0054564456805
:101B600025F0406545F080654560456C25F0406591
:101B700045F000654564456825F0405545F08055C1
:101B80004560456C25F0405545F000554564C568F5
:101B900025F0405545F00055C560C56C45F04055F1
:101BA000C564C56925F44025C561C56D45F440256A
:101BB000C5651501CD670D6E45F000750D6645686C
:101BC00025F4401545F480154560456C04E000009F
:101BD00000C0024000C0092025F4401545F400155E
:101BE0004564456825F4404545F480454560456CAD
:101BF00025F4404545F400454564456825F44025F5
:101C000045F480254560456C25F4402545F40025C4
:101C10004564456825F4403545F480354560456C9C
:101C200025F4403545F400354564456825F44055B4
:101C30004560456C25F4405545F400554564CE613A
:101C40000D6845F480050D60456825F440654560E4
:101C5000456C25F4406545F400654564CA610D682E
:101C600045F400150D60C56925F44015C561C56DC5
:101C700025F4401545F40015C565CF670D6E45F098
:101C800080650D66C56825F44065C560C56C25F4A2
:101C9000406545F40065C564CA630A6A22F400120F
:101CA0000A62426A22F0407242F000724262426E60
:101CB00022F0407242F000724266426A22F04062B4
:101CC00042F000624262426E22F0406242F00062E4
:101CD0004266826822F00C028260826C22F00C0262
:101CE00042F0080282640222CA630A6A42F00202D7
:101CF0000A62826822F003028260826C22F0030290
:101D000082640122CA630A6A22F001020A62C2687E
:101D100022F00302C260C26C22F00302921CC26471
:101D20001A02CA630A6A42F480320A62026922F421
:101D300040020261026D22F440020265C214CA65CB
:101D40000A6C22F400620A64026922F44012026101
:101D5000026D22F4401202650215CA650D6C25F46D
:101D600080650D64C56825F4400545F48005C560AF
:101D7000C56C25F4400545F40005C564C56825F02B
:101D8000C005C560C56C25F0C00545F08005C5647B
:101D90005502CD630E6A46F400260E62C66826F030
:101DA000C006C660C66C26F0C00646F08006C66453
:101DB000CD630D6A45F400250D62856825F44075F4
:101DC0008560856C25F4407545F400758564CC63A9
:101DD0000C6A44F010040C62846824F4403484607B
:101DE000846C24F4403444F4003484648B630B6AC0
:101DF00043F480730B62836823F040538360836CE9
:101E000023F0405383641301CB630B6A43F4804394
:101E10000B62836823F440138360836C23F44013C4
:101E200083648A63086A40F480600862F0BD000041
:101E3000FA4800214FF00112818001704170C0E921
:101E400002217047F5491C31002000F09FBB10B5FE
:101E5000F24C1434A288402A00D940228020216804
:101E600000F0C5FB216801442160A188081AA08008
:101E700010BD10B5E94C00201434216800F086FB39
:101E8000216801442160A188081AA08010BD0022A9
:101E90001146802000F0ABBBE149002000F076BB8A
:101EA00070B5DE48DD4D1C3005F11405007810F0EA
:101EB0001F040AD0D949DA4B01F11C004A78007995
:101EC000012C06D0022C26D109E0D448001D286040
:101ED0001DE002B3897888421DD2002015E000F091
:101EE0008F04200605D504F00F064FF48030B04073
:101EF00001E00120A0400AB922070CD18A68024201
:101F000009D0C9680142E8D0012018802B60FFF792
:101F10009EFF012070BD002070BD024670B5BF4815
:101F2000BE4C1C30017811F01F030146498804D0D3
:101F3000012B29D0022B27D111E0012924D132B164
:101F4000012000F0BDFAA08840F0020005E000206A
:101F500000F0B6FAA08820F00200A08021E000790D
:101F600000F08F00030605D500F00F034FF4803515
:101F70009D4001E00125854063782BB1030703D024
:101F8000A3682B4200D009B1002070BD22B100F03F
:101F9000E9FAE068284303E000F0EEFAE068A843BD
:101FA000E060012070BD9D4810B51C30007810F035
:101FB0001F0F9A4800F11C00C0782AD197491431AC
:101FC000012807D001F108020228937806D00328DF
:101FD0001FD112E093480860122012E092480022BC
:101FE00004E004780CB144882044521C9342F8D198
:101FF000027872B10860408803E08C481844086099
:1020000000788A88824200D98880FFF720FF01206B
:1020100010BD002010BD2DE9F84F804F00201C3767
:102020000090B8787D4E4FF000094FF0010A4FF450
:10203000803B00286BD07C4C65E06078022804D09F
:10204000042841D005285CD141E06179B87881420B
:1020500038D170702079B0707049002011F11001F2
:1020600001F80090401C0428FAD301254FEA060825
:102070000AFA05F0D8F80810084202D0284600F005
:102080005DFAD8F808100BFA05F0084203D045F0C5
:10209000800000F053FA6D1C102DE9D34FF00110B1
:1020A000C8E90209012000F00CFAE0794006B8F80E
:1020B000040002D540F0010001E020F00100A8F882
:1020C00004001EE060881DE0E078009019E00098B0
:1020D000B8B9A07800F08F05280604D505F00F01E7
:1020E0000BFA01F001E00AFA05F0B168014320465D
:1020F000B16000F0FCF9284600F016FA284600F01E
:1021000027FA207804442078002896D11FE086F82A
:10211000019001245546D846B16805FA04F00842FA
:1021200002D0204600F00AFAB16808FA04F008422A
:1021300003D044F0800000F001FA641C102CEBD3B3
:102140004FF00110C6E90209002000F0BAF9B87892
:102150007178884202D10120BDE8F88F0020FBE7AA
:102160002DE9FC5F2D4D00273E466878BB46B846FA
:10217000002871D0BA462C4C05F11C0968E0607843
:10218000022804D0042808D005285FD119E060791E
:10219000697888425AD0608859E0A77899F8041085
:1021A000E6784FF00008B94250D199F80200B042E9
:1021B0004CD11A484FF0010A103010F807B0C6553C
:1021C00044E099F80410B94240D1A17801F08F01A0
:1021D0000191090605D5019901F00F024FF48031F4
:1021E00001E0019A01219140009199F80200B0426A
:1021F0001ED1A8680843A860E9680098814320467A
:10220000E96000F074F9019800F08EF9019800F08F
:102210009FF9009948EA010818E00000E400001066
:10222000181D0010A8530000BA530000DB53000033
:102230005E450BD118EA010F08D1A8688843A86051
:10224000E8688843E860019800F078F92078044451
:102250002078002893D15046BDE8FC9F2DE9F0413D
:10226000494C0027A4F108062178A4F11C05082890
:1022700063D2DFE800F06204647262628381FFF778
:10228000E1FD2078C00900F04EF9E088B0802078A8
:10229000C0F34111F1BB61780C294AD2DFE801F0AB
:1022A0000609490B49101A1D1F253142FFF7F8FD99
:1022B0004DE0002000E00120FFF72FFE50B306E0C4
:1022C00010F01F0F35D1A07840F080002870BDE8D5
:1022D000F041DCE5FFF767FE39E000202AE010F06E
:1022E0001F0F26D128481B381AE010F01F0F20D1ED
:1022F000FFF791FE70B1FFF7CAFDBDE8F041FEF7B0
:1023000047B800F01F00012813D1687810B1207978
:10231000A97800E00DE088420BD21B490C39084433
:1023200030601CE000F01F00012802D1FFF718FF09
:10233000C4E7802000F016F9B780BDE8F0810806F8
:1023400008D4B0880028F8D0FFF793FDB0880028A3
:10235000EFD0F2E7BDE8F0419EE5080602D5BDE802
:10236000F04174E528780106E7D500F07F00287079
:10237000BDE8F04100F054B8802000E00020BDE846
:10238000F04100F0F9B8000000010010014600071C
:10239000C00E090600D5401C7047DA491022C1F86A
:1023A0000822C1F8100200BFD1F80002C006FBD518
:1023B0007047D44A1023C2F80832C2F8100200BF96
:1023C000D2F80002C006FBD5C2F80832C2F81012DB
:1023D000D2F80002C006FBD57047CA493022C1F8C6
:1023E0000822C1F8100200BFD1F800028006FBD518
:1023F000D1F81402704710B5040001D0012000E0AC
:1024000000204FF4807141EA0041BF48FFF7D1FF3F
:10241000BE494FF000700CB1886710BDC86710BD91
:1024200030B5BB49BB4D41EA004421462846FFF781
:10243000C0FF21462846BDE83040BAE7B148002138
:10244000C0F848124021C0F84C120122C0F84822BE
:10245000C0F84C12D0F80012C905FBD54FF0FF317F
:10246000C0F83812C0F83412C0F808120C21C0F8B5
:1024700004127047A84800B5C16821F0405141F0EE
:102480000051C160C16C41F04051C164A3491A20A0
:102490000860091D0A6830EA0202FBD14FF0E02112
:1024A0004FF08070C1F880029D4B202283F80024F9
:1024B000C1F80001FFF7C2FF00205DF804EBAFE7B1
:1024C000704710B500B101204FF4807444EA004118
:1024D0009448FFF76EFF8B480321C0F8441200BFF9
:1024E000D0F80012C905FBD5C0F8084210BD10B5E0
:1024F00002468078FFF74AFF8249D1F8443201242E
:1025000084402343C1F84432C1F848029088C1F89E
:102510004C0200BFD1F80002C005FBD54FF480701B
:10252000C1F8080210BD704700B5FFF72FFF7E49C4
:102530005DF804EB41EA004089133AE700B5FFF784
:1025400025FF79495DF804EB41EA0040774930E71F
:1025500000B5FFF71BFF74495DF804EB41EA00404A
:10256000891326E700B5FFF711FF6F495DF804EB0B
:1025700041EA00406E491CE700B5FFF707FF6A49D2
:102580005DF804EB41EA0040891312E700F00F0206
:10259000012370B503EB82035A4AC2F8283200BF08
:1025A000D2F820321C05FBD5C3F309030024DD1C3F
:1025B00005E000BFD2F8186241F8046B641CB4EB6C
:1025C000950FF7D30021C2F8281241F24821C140EB
:1025D000C9070AD1FFF7DAFE4FF4A06141EA0040D3
:1025E000FFF7DBFE5348FFF7D8FE184670BD70B505
:1025F00013460546434C00F00F00022202EB800018
:10260000C4F82802C4F824320020DA1C05E000BF18
:1026100051F8046BC4F81C62401CB0EB920FF7D366
:102620000020C4F828022846FFF7B0FE4FF4A0614E
:1026300041EA0040FFF7B1FE3F48FFF7AEFE184603
:1026400070BD2DE9F0412F4DD5F80032C5F80832A4
:10265000180721D52C48FFF7A0FE3848FFF7BDFE2C
:10266000C10605D5FFF7EAFEBDE8F041FDF781BEE2
:10267000810705D5BDE8F04100F00100FDF773BE0C
:10268000010709D5400703D5BDE8F041FDF778BE45
:10269000BDE8F041FDF77BBE294E58074FF001071A
:1026A0001CD4BDE8F0810024D5F8302207FA04F1EB
:1026B0000A4210D06008C5F8381200BFD5F80012E1
:1026C0008906FBD5D5F81412E2070CD056F8201075
:1026D00009B103208847641C202CE5D3D5F83002CB
:1026E0000028E0D1DDE73CB9490705D5316819B1CB
:1026F000012088470124D7E756F820100029EAD0A6
:102700000220E7E700C000500005FE0000C00920DD
:10271000000180000005D00000C00240F4CF00504E
:1027200018E000E00005D80000054000000120008E
:10273000000101000005F2000005FA000002FE00A1
:102740004C54000019480621016107210160002155
:102750004161416202214160C168C906FCD400E0C8
:102760008168C1684907FBD4002070470F49886021
:10277000C868C006FCD48868704700B50B4602469E
:1027800004E000BF12F8010BFFF7F0FF5B1EF9D267
:1027900000BD00B50B46024604E00020FFF7E6FF4F
:1027A00002F8010B5B1EF8D200BD0000008008405B
:1027B0002DE9F047F74E80464FF080773068BC1126
:1027C000F54DB84249D100BF00BF00BF00BF00BFF8
:1027D00000BF00BF00BF00BF00BF00BF00BF00BF01
:1027E00000BF00BF00BF00BF00BF00BF00BF00BFF1
:1027F00000BF00BF00BF00BF00BF00BF00BF00BFE1
:1028000000BF00BF00BFEC631520FFF7AFFF002043
:10281000FFF7ACFF00F0FF09AC6300BF00BF00BFD3
:1028200000BF00BF00BF00BF00BF00BF00BF00BFB0
:1028300000BF00BF00BF00BF00BF00BF00BF00BFA0
:1028400000BF00BF00BF00BF00BF00BF00BF00BF90
:1028500000BF00BF00BF00BF00BF00BF00BF00BF80
:1028600000BF00BF00BF00BF00BF00BF00BF00BF70
:1028700000BF00BF00BF00BF00BF00BF00BF00BF60
:1028800000BF00BF00BF00BF00BF00BF00BF00BF50
:1028900000BF00BF00BF00BF00BFEC630620FFF712
:1028A00065FFAC6300BF00BF00BF00BF00BF00BF3B
:1028B00000BF00BF00BF00BF00BF00BF00BF00BF20
:1028C00000BF00BF00BF00BF00BF00BF00BF00BF10
:1028D00000BF00BF00BF00BF00BF00BF00BF00BF00
:1028E00000BF00BF00BF00BF00BF00BF00BF00BFF0
:1028F00000BF00BF00BF00BF00BF00BF00BF00BFE0
:1029000000BF00BF00BF00BF00BF00BF00BF00BFCF
:1029100000BF00BF00BF00BF00BF00BF00BF00BFBF
:1029200000BF00BFEC630120FFF720FF4FEA8800E3
:10293000FFF71CFF3068B84202D14846FFF716FF88
:10294000AC6300BF00BF00BF00BF00BF00BF00BF3F
:1029500000BF00BF00BF00BF00BF00BF00BF00BF7F
:1029600000BF00BF00BF00BF00BF00BF00BF00BF6F
:1029700000BF00BF00BF00BF00BF00BF00BF00BF5F
:1029800000BFBDE8F0872DE9FC5F8846044601A939
:10299000824800F05DFB824D824E834FF0BB0320E6
:1029A0008DF8000020098DF8010020018DF802004B
:1029B0004FF000098DF8039000BF00BF00BF00BFBB
:1029C00000BF00BF00BF00BF00BF00BF00BF00BF0F
:1029D00000BF00BF00BF00BF00BF00BF00BF00BFFF
:1029E00000BF00BF00BF00BF00BF00BF00BF00BFEF
:1029F00000BF00BF00BF00BFDFF89CB14FF4802ACA
:102A0000CBF83CA004216846FFF7B7FE0024002065
:102A1000FFF7ACFEC0B28DF8040000E003E018F848
:102A20000410884208D08220286022203060784636
:102A300038608220BDE8FC9F641CB4F5805FE6D35B
:102A4000CBF838A000BF00BF00BF00BF00BF00BF71
:102A500000BF00BF00BF00BF00BF00BF00BF00BF7E
:102A600000BF00BF00BF00BF00BF00BF00BF00BF6E
:102A700000BF00BF00BF00BF00BF00BF00BF00BF5E
:102A800000BF00BFC5F800907846C6F800903860D7
:102A90000020CFE72DE9F0474FF0000900BF00BF4D
:102AA00000BF00BF00BF00BF00BF00BF00BF00BF2E
:102AB00000BF00BF00BF00BF00BF00BF00BF00BF1E
:102AC00000BF00BF00BF00BF00BF00BF00BF00BF0E
:102AD00000BF00BF00BF00BF00BF00BF2E4E4FF4BD
:102AE0008025F5639F20FFF741FE0020FFF73EFEA3
:102AF00000F0FF080020FFF739FEC4B20020FFF706
:102B000035FEC1B2B56300BF00BF00BF00BF00BF4C
:102B100000BF00BF00BF00BF00BF00BF00BF00BFBD
:102B200000BF00BF00BF00BF00BF00BF00BF00BFAD
:102B300000BF00BF00BF00BF00BF00BF00BF00BF9D
:102B400000BF00BF00BF164D164E174FB8F1C20FA1
:102B500001D1202C07D082202860212030607846C7
:102B6000386082200DE70B4814291FD0152920D08A
:102B7000162922D0182923D0C0F800900020FFF792
:102B800017FEC5F800907846C6F80090386000201F
:102B9000F7E600001001001000C00920A086010027
:102BA0006C00001070000010740000104FF48011D1
:102BB00001E04FF400110160E0E74FF48001FAE713
:102BC0004FF08071F7E72DE9F34FC3B08046002442
:102BD0004FF0820AFE4DFF4EFF4F4FF0210BA146F2
:102BE00041A9FE4800F034FA00286CD100F09CFAAC
:102BF00002208DF800004FEA18108DF8010004EB58
:102C000008108DF8020044988DF8039000EB042121
:102C10004FF4807201A801F08FFF00BF00BF00BF1A
:102C200000BF00BF00BF00BF00BF00BF00BF00BFAC
:102C300000BF00BF00BF00BF00BF00BF00BF00BF9C
:102C400000BF00BF00BF00BF00BF00BF00BF00BF8C
:102C500000BF00BF00BF00BF00BFE1494FF48020AC
:102C6000C8634FF482716846FFF787FDDC494FF473
:102C70008020886300BF00BF00BF00BF00BF00BF4F
:102C800000BF00BF00BF00BF00BF00BF00BF00BF4C
:102C900000BF00BF00BF00BF00BF00BF00BF00BF3C
:102CA00000BF00BF00BF00BF00BF00BF00BF00BF2C
:102CB00000BF00BF641CE4B2102C91D341A9C748E7
:102CC00000F0C6F948B1C5F800A07846C6F800B0D3
:102CD0003860822045B0BDE8F08F00F06FFAC5F88B
:102CE00000907846C6F8009038600020F2E72DE9A1
:102CF000F04F89B0DFF8D8825FEA020B4FF0000690
:102D000007910FD04FF4805501462A466846FDF7DB
:102D100053FBDDE90047284601F0B8FE5FEA0009F1
:102D20000CD016E08621AB48C8F8001009210160DC
:102D30007946A9480160862009B0CCE78221A548E0
:102D4000C8F80010222101607946A3480160822062
:102D5000F2E7ABEB0605C7F580504FF0000AA8423A
:102D600000D20546B5F5805F04D02046494600F004
:102D7000A3FCD8B907982A46811907EB090001F08E
:102D8000DBFE204600F01DFC80B920464946FFF7D7
:102D90001AFF58B920464946FFF7F5FD78B10AF108
:102DA000010000F0FF0ABAF1030F05D3484601F015
:102DB0009CFED8F80000BFE7BAF1000FE1D12E4425
:102DC0000027641C5E45C4D3484601F08EFE81494D
:102DD0000020C8F80000086079467F4801600020A4
:102DE000AAE72DE9FF4F8DB00D46DDF8689000266B
:102DF000774C07935FEA09013FD04FF480570146B3
:102E00003A466846FDF7D8FADDE900B10C913A463A
:102E1000691C6846FDF7D0FADDE90010CDE9040130
:102E20003A4668460F99FDF7C7FADDE9008500BF0D
:102E3000A9EB0607C5F58050B84200D2074625B178
:102E4000D8457CD10C98854279D14FF4805001F05F
:102E50001DFE5FEA000A1BD0D8454FD10C98854271
:102E60004CD12A464FEA0830514600F0FEFA0006DF
:102E700018D5504601F039FE79E08620206055488B
:102E800009210160784654490860862011B022E784
:102E9000822020604F482221016079464E4801601F
:102EA0008220F3E70598804509D1049901EB0030B1
:102EB000C1F58052514400F0D8FA0006D9D44046FA
:102EC00000F07FFB0006D4D407983A46811905EB41
:102ED0000A0001F031FEEA194FEA0830514601F0CC
:102EE000DCF90006C5D40599884533D1049800EB78
:102EF00001300499C1F58052514427E00599884575
:102F00000AD1049800EB01300499C1F58052514672
:102F100000F0ABFA0006ACD4404600F052FB0006CD
:102F2000A7D407983A4681190F98304401F0B5F9B3
:102F300000069ED4059988450CD1049800E00DE068
:102F400000EB01300499C1F58052514601F0A5F91A
:102F500000068ED4504601F0C8FD0AE007983A46B4
:102F600081190F98304401F098F9000601D52068C6
:102F70008CE73E44002508F101084E45FFF458AFA8
:102F8000144900202060086078461349086000203A
:102F90007CE71448006870474FF4805070472DE973
:102FA000F04FDFF82C80DFF82CB089B00F0004461A
:102FB0004FF0000633D04FF4805501462A4668464C
:102FC000FDF7FAF9DDE900A105912A4621460BE05B
:102FD0006C0000107000001074000010A08601004A
:102FE00000C009201001001006A8FDF7E5F9DDE991
:102FF00006404FF00009BD1BC0F58051A94200D228
:103000000D4620B1544515D10599884212D120466C
:1030100000F0D7FA00060DD5D8F800008CE686211E
:10302000C8F800100921CBF8001079463B48016030
:10303000862081E62E44641C4846BE42DBD3C8F895
:1030400000007946CBF8000034480160002073E6A8
:103050002DE9F041324C0F460646A56806E0A0680F
:10306000401BB04202D30120BDE8F081384600F099
:1030700003F80028F3D1F7E770B5044600BF00BF9E
:1030800000BF00BF00BF00BF00BF00BF00BF00BF48
:1030900000BF00BF00BF00BF00BF00BF00BF00BF38
:1030A00000BF00BF00BF00BF00BF00BF00BF00BF28
:1030B00000BF00BF00BF00BF00BF00BF194E4FF4EC
:1030C0008025F5630520FFF751FB0020FFF74EFB3D
:1030D0002070B56300BF00BF00BF00BF00BF00BFCE
:1030E00000BF00BF00BF00BF00BF00BF00BF00BFE8
:1030F00000BF00BF00BF00BF00BF00BF00BF00BFD8
:1031000000BF00BF00BF00BF00BF00BF00BF00BFC7
:1031100000BF00BF207800F0010070BD74000010F7
:103120000080004000C0092070B500BF00BF00BF94
:1031300000BF00BF00BF00BF00BF00BF00BF00BF97
:1031400000BF00BF00BF00BF00BF00BF00BF00BF87
:1031500000BF00BF00BF00BF00BF00BF00BF00BF77
:1031600000BF00BF00BF00BF00BFFE4C4FF4802572
:10317000E5630620FFF7FAFAA56300BF00BF00BFB2
:1031800000BF00BF00BF00BF00BF00BF00BF00BF47
:1031900000BF00BF00BF00BF00BF00BF00BF00BF37
:1031A00000BF00BF00BF00BF00BF00BF00BF00BF27
:1031B00000BF00BF00BF00BF00BF70BD70B500BF43
:1031C00000BF00BF00BF00BF00BF00BF00BF00BF07
:1031D00000BF00BF00BF00BF00BF00BF00BF00BFF7
:1031E00000BF00BF00BF00BF00BF00BF00BF00BFE7
:1031F00000BF00BF00BF00BF00BF00BF00BFD94C71
:103200004FF48025E5630420FFF7B0FAA56300BF03
:1032100000BF00BF00BF00BF00BF00BF00BF00BFB6
:1032200000BF00BF00BF00BF00BF00BF00BF00BFA6
:1032300000BF00BF00BF00BF00BF00BF00BF00BF96
:1032400000BF00BF00BF00BF00BF00BF00BF70BD18
:1032500070B5064600BF00BF00BF00BF00BF00BF83
:1032600000BF00BF00BF00BF00BF00BF00BF00BF66
:1032700000BF00BF00BF00BF00BF00BF00BF00BF56
:1032800000BF00BF00BF00BF00BF00BF00BF00BF46
:1032900000BF00BFB34D4FF48024EC635020FFF714
:1032A00065FAAC6300BF00BF00BF00BF00BF00BF36
:1032B00000BF00BF00BF00BF00BF00BF00BF00BF16
:1032C00000BF00BF00BF00BF00BF00BF00BF00BF06
:1032D00000BF00BF00BF00BF00BF00BF00BF00BFF6
:1032E00000BF00BF00BF00BF00BF00BF00BF00BFE6
:1032F00000BF00BF00BF00BF00BF00BF00BF00BFD6
:1033000000BF00BF00BF00BF00BF00BF00BF00BFC5
:1033100000BF00BF00BF00BF00BF00BF00BF00BFB5
:1033200000BF00BFEC630120FFF720FAB000FFF7F9
:103330001DFAAC6300BF00BF00BF00BF00BF00BFED
:1033400000BF00BF00BF00BF00BF00BF00BF00BF85
:1033500000BF00BF00BF00BF00BF00BF00BF00BF75
:1033600000BF00BF00BF00BF00BF00BF00BF00BF65
:1033700000BF00BF70BD2DE9FE430F46044602A901
:10338000794800F0BCFD794D794EDFF8E88148B10D
:10339000822028602220794630608220C8F8001000
:1033A000BDE8FE839DF80800800701D4FFF7BCFE4E
:1033B00002208DF80000200C8DF80100200A8DF805
:1033C00002008DF803408DF8047000BF00BF00BFFD
:1033D00000BF00BF00BF00BF00BF00BF00BF00BFF5
:1033E00000BF00BF00BF00BF00BF00BF00BF00BFE5
:1033F00000BF00BF00BF00BF00BF00BF00BF00BFD5
:1034000000BF00BF00BF00BF00BF564F4FF4802475
:10341000FC6305216846FFF7B0F9BC6300BF00BF3D
:1034200000BF00BF00BF00BF00BF00BF00BF00BFA4
:1034300000BF00BF00BF00BF00BF00BF00BF00BF94
:1034400000BF00BF00BF00BF00BF00BF00BF00BF84
:1034500000BF00BF00BF00BF00BF00BF002028604A
:1034600079463060C8F800109AE72DE9FC5F3F4DBF
:103470003F4E404F5FEA020A8B4604464FF0000879
:103480000DD001A9384800F03AFD80B182202860B3
:1034900021203060784638608220BDE8FC9FC5F866
:1034A00000807846C6F8008038600020F5E70320E9
:1034B0008DF80000200C8DF80100200A8DF8020024
:1034C0008DF8034000BF00BF00BF00BF00BF00BFBA
:1034D00000BF00BF00BF00BF00BF00BF00BF00BFF4
:1034E00000BF00BF00BF00BF00BF00BF00BF00BFE4
:1034F00000BF00BF00BF00BF00BF00BF00BF00BFD4
:1035000000BF00BF174C4FF48029C4F83C90042141
:103510006846FFF732F951465846FFF73AF9C4F8C2
:10352000389000BF00BF00BF00BF00BF00BF00BF9A
:1035300000BF00BF00BF00BF00BF00BF00BF00BF93
:1035400000BF00BF00BF00BF00BF00BF00BF00BF83
:1035500000BF00BF00BF00BF00BF00BF00BF00BF73
:1035600000BF9CE700C00920A08601006C0000108D
:1035700070000010740000102DE9F05FFF4EDFF8BE
:103580000094DFF800A4150083460F464FF00008B2
:103590000ED000240AE0395D0BEB0400FFF7EBFED0
:1035A000000602D53068BDE8F09F641CAC42F2D33F
:1035B000C6F800807946C9F800800020CAF80010DB
:1035C000F1E72DE9FC47044601A9EF4800F097FC1C
:1035D000EA4DEB4EDFF8AC9348B182202860222000
:1035E000794630608220C9F80010BDE8FC879DF85C
:1035F0000400800701D4FFF797FD20208DF800001C
:1036000020098DF8010020018DF8020000248DF8BA
:10361000034000BF00BF00BF00BF00BF00BF00BF2E
:1036200000BF00BF00BF00BF00BF00BF00BF00BFA2
:1036300000BF00BF00BF00BF00BF00BF00BF00BF92
:1036400000BF00BF00BF00BF00BF00BF00BF00BF82
:1036500000BFDFF838834FF48027C8F83C7004219E
:103660006846FFF78AF8C8F8387000BF00BF00BF8F
:1036700000BF00BF00BF00BF00BF00BF00BF00BF52
:1036800000BF00BF00BF00BF00BF00BF00BF00BF42
:1036900000BF00BF00BF00BF00BF00BF00BF00BF32
:1036A00000BF00BF00BF00BF00BF2C607946346080
:1036B0000020C9F8001098E72DE9FC478A46044627
:1036C00001A9B14800F01BFCAC4DAD4EDFF8B4923F
:1036D00040B1822028602220794630608220C9F8DB
:1036E000001082E703208DF8000020098DF801000A
:1036F00020018DF8020000248DF8034000BF00BFB8
:1037000000BF00BF00BF00BF00BF00BF00BF00BFC1
:1037100000BF00BF00BF00BF00BF00BF00BF00BFB1
:1037200000BF00BF00BF00BF00BF00BF00BF00BFA1
:1037300000BF00BF00BF00BF00BF00BFDFF84C826A
:103740004FF48027C8F83C7004216846FFF715F84D
:10375000B9115046FFF71DF8C8F8387000BF00BF18
:1037600000BF00BF00BF00BF00BF00BF00BF00BF61
:1037700000BF00BF00BF00BF00BF00BF00BF00BF51
:1037800000BF00BF00BF00BF00BF00BF00BF00BF41
:1037900000BF00BF00BF00BF00BF00BF2C60794664
:1037A00034600020C9F800101FE72DE9F34F83B003
:1037B000044601A9744800F0A2FB704D704E714F91
:1037C0004FF0820818B12120C5F800806CE09DF808
:1037D0000400800701D4FFF7A7FCAD208DF800009E
:1037E00020098DF8010020018DF802004FF0000B38
:1037F0008DF803B000BF00BF00BF00BF00BF00BF17
:1038000000BF00BF00BF00BF00BF00BF00BF00BFC0
:1038100000BF00BF00BF00BF00BF00BF00BF00BFB0
:1038200000BF00BF00BF00BF00BF00BF00BF00BFA0
:1038300000BF00BFDFF854914FF4802A5446C9F806
:103840003CA004216846FEF798FF02210498FEF789
:1038500094FFC9F8384000BF00BF00BF00BF00BFE1
:1038600000BF00BF00BF00BF00BF00BF00BF00BF60
:1038700000BF00BF00BF00BF00BF00BF00BF00BF50
:1038800000BF00BF00BF00BF00BF00BF00BF00BF40
:1038900000BF00BF00BF022401A93B4800F02FFB7E
:1038A00048B12220C5F80080306078463860822018
:1038B00005B0BDE8F08F00BF00BF00BF00BF00BF74
:1038C00000BF00BF00BF00BF00BF00BF00BF00BF00
:1038D00000BF00BF00BF00BF00BF00BF00BF00BFF0
:1038E00000BF00BF00BF00BF00BF00BF00BF00BFE0
:1038F00000BF00BF00BFC9F83CA0AD20FEF736FFF7
:10390000049802212044FEF738FFC9F838A000BF10
:1039100000BF00BF00BF00BF00BF00BF00BF00BFAF
:1039200000BF00BF00BF00BF00BF00BF00BF00BF9F
:1039300000BF00BF00BF00BF00BF00BF00BF00BF8F
:1039400000BF00BF00BF00BF00BF00BF00BFA41C7E
:10395000A4B2B4F5805F9FD301A90B4800F0CFFA61
:1039600000287FF430AFFFF729FCC5F800B0784697
:10397000C6F800B0386000209AE700006C00001024
:103980007000001074000010A086010000C0092023
:1039900070B5FD4DFD4EFE4C2AB1FFF766FD0006E9
:1039A00009D5206870BD86202060092028607846EF
:1039B0003060862070BD002020602860784630602E
:1039C000002070BD2DE9F04F89B0DFF8C483DFF827
:1039D000B8B35FEA02094FF0000607910FD04FF429
:1039E000805501462A466846FCF7E6FCDDE90047BB
:1039F000284601F04BF85FEA000A0CD016E0862159
:103A0000C8F800100921CBF800107946DF480160A2
:103A1000862009B04DE78221C8F800102221CBF89A
:103A200000107946D94801608220F2E7A9EB06052B
:103A3000C7F58050A84200D20546B5F5805F04D096
:103A400020465146FFF738FE80B92046FFF7B9FD02
:103A500060B907982A46811907EB0A0001F06CF853
:103A60002E4420465146FFF7A0FE28B1504601F0F3
:103A70003CF8D8F80000CCE70027641C4E45D5D3AD
:103A8000504601F032F80020C8F800007946CBF823
:103A90000000BE4801600020BBE72DE9FF4F8DB05C
:103AA0000D46DDF868900026B94C07935FEA0901DE
:103AB0003FD04FF4805701463A466846FCF77CFCFD
:103AC000DDE900B10C913A46691C6846FCF774FCCC
:103AD000DDE90010CDE904013A4668460F99FCF78C
:103AE0006BFCDDE9008500BFA9EB0607C5F580503A
:103AF000B84200D2074625B1D8457CD10C98854202
:103B000079D14FF4805000F0C1FF5FEA000A1BD06A
:103B1000D8454FD10C9885424CD12A464FEA0830FF
:103B20005146FFF7A2FC000618D5504600F0DDFF15
:103B300079E0862020609448092101607846934905
:103B40000860862011B0B4E6822020608E482221D1
:103B5000016079468D4801608220F3E70598804531
:103B600009D1049901EB0030C1F580525144FFF7AF
:103B70007CFC0006D9D44046FFF723FD0006D4D4D0
:103B800007983A46811905EB0A0000F0D5FFEA19BB
:103B90004FEA08305146FFF7EFFC0006C5D40599FF
:103BA000884533D1049800EB01300499C1F5805267
:103BB000514427E0059988450AD1049800EB01306B
:103BC0000499C1F580525146FFF74FFC0006ACD472
:103BD0004046FFF7F6FC0006A7D407983A4681193D
:103BE0000F983044FFF7C8FC00069ED4059988451D
:103BF0000CD1049800E00DE000EB01300499C1F510
:103C000080525146FFF7B8FC00068ED4504600F0B3
:103C10006CFF0AE007983A4681190F983044FFF785
:103C2000ABFC000601D520688CE73E44002508F176
:103C300001084E45FFF458AF53490020206008604A
:103C400078465249086000207CE72DE9F0474FF0A4
:103C5000000900BF00BF00BF00BF00BF00BF00BF22
:103C600000BF00BF00BF00BF00BF00BF00BF00BF5C
:103C700000BF00BF00BF00BF00BF00BF00BF00BF4C
:103C800000BF00BF00BF00BF00BF00BF00BF00BF3C
:103C900000BF404E4FF48025F5639F20FEF766FD80
:103CA0000020FEF763FD00F0FF080020FEF75EFD38
:103CB000C4B20020FEF75AFDC1B2B56300BF00BF19
:103CC00000BF00BF00BF00BF00BF00BF00BF00BFFC
:103CD00000BF00BF00BF00BF00BF00BF00BF00BFEC
:103CE00000BF00BF00BF00BF00BF00BF00BF00BFDC
:103CF00000BF00BF00BF00BF00BF00BF244D224E69
:103D0000224FB8F1BF0F03D1252C0AD0262C08D0A2
:103D10008220286021203060784638608220BDE80B
:103D2000F0871D48412912D04FF48002422912D059
:103D30004A2910D0C0F800900020FFF789FAC5F892
:103D400000907846C6F8009038600020E7E74FF40E
:103D500000110160F0E70260EEE72DE9F84F6946D7
:103D60000E4800F0CCF88227094C074D074E4FF063
:103D7000220A002862D19DF80000800701D4FFF7D5
:103D8000D3F900BF00BF0BE07000001074000010FA
:103D90006C00001000C0092014010010A086010072
:103DA00000BF00BF00BF00BF00BF00BF00BF00BF1B
:103DB00000BF00BF00BF00BF00BF00BF00BF00BF0B
:103DC00000BF00BF00BF00BF00BF00BF00BF00BFFB
:103DD00000BF00BF00BF00BF00BF00BFDFF8EC9115
:103DE0004FF48028C9F83C806020FEF7BFFCC9F87A
:103DF000388000BF00BF00BF00BF00BF00BF00BFD2
:103E000000BF00BF00BF00BF00BF00BF00BF00BFBA
:103E100000BF00BF00BF00BF00BF00BF00BF00BFAA
:103E200000BF00BF00BF00BF00BF00BF00BF00BF9A
:103E300000BF6946664800F062F838B127607846EE
:103E4000C5F800A030608220BDE8F88F0020206017
:103E50002860784630600020F6E75E4800687047CA
:103E60004FF4805070472DE9F04FDFF86C81DFF898
:103E70006CB189B00F0004464FF0000626D04FF415
:103E8000805501462A466846FCF796FADDE900A10E
:103E900005912A46214606A8FCF78EFADDE9064080
:103EA0004FF00009BD1BC0F58051A94200D20D465C
:103EB00020B1544515D10599884212D12046FFF70B
:103EC00080FB00060DD5D8F80000A2E58621C8F8D1
:103ED00000100921CBF80010794641480160862086
:103EE00097E52E44641C4846BE42DBD3C8F8000068
:103EF0007946CBF800003A480160002089E52DE9B9
:103F0000F041384C0F460646A56806E0A068401B05
:103F1000B04202D30120BDE8F081384600F003F83A
:103F20000028F3D1F7E770B5044600BF00BF00BF1B
:103F300000BF00BF00BF00BF00BF00BF00BF00BF89
:103F400000BF00BF00BF00BF00BF00BF00BF00BF79
:103F500000BF00BF00BF00BF00BF00BF00BF00BF69
:103F600000BF00BF00BF00BF00BF184E4FF4802548
:103F7000F5630520FEF7FAFB0020FEF7F7FB207043
:103F8000B56300BF00BF00BF00BF00BF00BF00BFE0
:103F900000BF00BF00BF00BF00BF00BF00BF00BF29
:103FA00000BF00BF00BF00BF00BF00BF00BF00BF19
:103FB00000BF00BF00BF00BF00BF00BF00BF00BF09
:103FC00000BF207800F0010070BD000000C0092093
:103FD00020A10700140100106C00001070000010F8
:103FE00074000010008000402DE9FF4703A9FE483F
:103FF00000F063FBFD4DFE4EDFF8F89350B18220D8
:1040000028602120794630608220C9F8001004B071
:10401000BDE8F0879DF80C00800701D4FFF784F815
:1040200042208DF800000024CDF80140CDF8054075
:10403000ADF8094000BF00BF00BF00BF00BF00BF18
:1040400000BF00BF00BF00BF00BF00BF00BF00BF78
:1040500000BF00BF00BF00BF00BF00BF00BF00BF68
:1040600000BF00BF00BF00BF00BF00BF00BF00BF58
:1040700000BF00BFDFF880834FF48027C8F83C7092
:104080000B216846FEF779FBC8F8387000BF00BF07
:1040900000BF00BF00BF00BF00BF00BF00BF00BF28
:1040A00000BF00BF00BF00BF00BF00BF00BF00BF18
:1040B00000BF00BF00BF00BF00BF00BF00BF00BF08
:1040C00000BF00BF00BF00BF00BF00BF2C6079462B
:1040D00034600020C9F8001099E72DE9F34F85B04E
:1040E000044603A9C04800F0E8FAC04DC04EC14FD5
:1040F0004FF0820B18B12120C5F800B060E0FFF747
:1041000013F842208DF800004FF0000ACDF801A00E
:10411000CDF805A0ADF809A000BF00BF00BF00BFEB
:1041200000BF00BF00BF00BF00BF00BF00BF00BF97
:1041300000BF00BF00BF00BF00BF00BF00BF00BF87
:1041400000BF00BF00BF00BF00BF00BF00BF00BF77
:1041500000BF00BF00BF00BFDFF89C924FF4802873
:10416000C9F83C800B216846FEF707FBC9F8388088
:1041700000BF00BF00BF00BF00BF00BF00BF00BF47
:1041800000BF00BF00BF00BF00BF00BF00BF00BF37
:1041900000BF00BF00BF00BF00BF00BF00BF00BF27
:1041A00000BF00BF00BF00BF00BF00BF00BF00BF17
:1041B00003A98D4800F081FA48B12220C5F800B06B
:1041C000306078463860822007B0BDE8F08F9DF8F7
:1041D0000C00800701D4FEF7A7FF02208DF8000035
:1041E000200C8DF80100200A8DF8020006988DF849
:1041F00003408DF8040000BF00BF00BF00BF00BF38
:1042000000BF00BF00BF00BF00BF00BF00BF00BFB6
:1042100000BF00BF00BF00BF00BF00BF00BF00BFA6
:1042200000BF00BF00BF00BF00BF00BF00BF00BF96
:1042300000BF00BF00BF4446C846C9F83C40052146
:104240006846FEF79AFAC8F8384000BF00BF00BFC2
:1042500000BF00BF00BF00BF00BF00BF00BF00BF66
:1042600000BF00BF00BF00BF00BF00BF00BF00BF56
:1042700000BF00BF00BF00BF00BF00BF00BF00BF46
:1042800000BF00BF00BF00BF00BFC5F800A0784658
:10429000C6F800A03860002096E72DE9F05F534E85
:1042A000DFF84C91DFF84CA1150083460F464FF024
:1042B00000080ED000240AE0395D0BEB0400FFF784
:1042C0000CFF000602D53068BDE8F09F641CAC42CC
:1042D000F2D3C6F800807946C9F800800020CAF8F9
:1042E0000010F1E72DE9F34F0024404D404E414FBF
:1042F000C3B080464FF0820A4FF0210BA14641A97E
:10430000394800F0DAF900287CD19DF804018007D3
:1043100001D4FEF709FF02208DF800004FEA1810C3
:104320008DF8010004EB08108DF8020044988DF818
:10433000039000EB04214FF4807201A800F0FCFB15
:1043400000BF00BF00BF00BF00BF00BF00BF00BF75
:1043500000BF00BF00BF00BF00BF00BF00BF00BF65
:1043600000BF00BF00BF00BF00BF00BF00BF00BF55
:1043700000BF00BF00BF00BF00BF00BF00BF00BF45
:104380001D494FF48020C8634FF482716846FEF7E0
:10439000F4F919494FF48020886300BF00BF00BFC3
:1043A00000BF00BF00BF00BF00BF00BF00BF00BF15
:1043B00000BF00BF00BF00BF00BF00BF00BF00BF05
:1043C00000BF00BF00BF00BF00BF00BF00BF00BFF5
:1043D00000BF00BF00BF00BF00BF641CE4B2102CD0
:1043E0008DD341A900480AE0A08601006C000010AE
:1043F000700000107400001000C0092002E000F0FE
:104400005CF940B1C5F800A07846C6F800B0386045
:10441000822045B0D9E6FEF7D1FEC5F80090784677
:10442000C6F8009038600020F3E72DE9F04F89B01E
:10443000DFF85483DFF854B35FEA02094FF0000657
:1044400007910FD04FF4805501462A466846FBF786
:10445000B3FFDDE90047284600F018FB5FEA000AD9
:104460000CD016E08621C8F800100921CBF8001006
:104470007946C7480160862009B0A6E68221C8F8BF
:1044800000102221CBF800107946C148016082203B
:10449000F2E7A9EB0605C7F58050A84200D2054611
:1044A000B5F5805F04D020465146FFF705F980B985
:1044B0002046FFF786F860B907982A46811907EB6E
:1044C0000A0000F039FB2E4420465146FFF70AFF50
:1044D00028B1504600F009FBD8F80000CCE70027CF
:1044E000641C4E45D5D3504600F0FFFA0020C8F8B2
:1044F00000007946CBF80000A54801600020BBE72A
:104500002DE9FF4F8DB00D46DDF8689000269E4CDA
:1045100007935FEA09013ED04FF4805701463A46BF
:104520006846FBF749FFDDE900B10C913A46691C8A
:104530006846FBF741FFDDE90010CDE904013A468A
:1045400068460F99FBF738FFDDE90085A9EB060700
:10455000C5F58050B84200D2074625B1D8457CD178
:104560000C98854279D14FF4805000F08FFA5FEAC1
:10457000000A1BD0D8454FD10C9885424CD12A4611
:104580004FEA08305146FEF770FF000618D5504636
:1045900000F0ABFA79E0862020607C4809210160B8
:1045A00078467B490860862011B00EE682202060A4
:1045B0007648222101607946754801608220F3E740
:1045C0000598804509D1049901EB0030C1F580526E
:1045D0005144FEF74AFF0006D9D44046FEF7F1FFEA
:1045E0000006D4D407983A46811905EB0A0000F07A
:1045F000A3FAEA194FEA08305146FFF74EFE0006CB
:10460000C5D40599884533D1049800EB013004994D
:10461000C1F58052514427E0059988450AD1049894
:1046200000EB01300499C1F580525146FEF71DFFA1
:104630000006ACD44046FEF7C4FF0006A7D4079896
:104640003A4681190F983044FFF727FE00069ED4A2
:10465000059988450CD1049800E00DE000EB01308D
:104660000499C1F580525146FFF717FE00068ED41B
:10467000504600F03AFA0AE007983A4681190F9836
:104680003044FFF70AFE000601D520688CE73E445F
:10469000002508F101084E45FFF458AF3B490020C2
:1046A0002060086078463A49086000207CE74FF4B3
:1046B000800070474FF4805070472DE9F041354C31
:1046C0000F460646A56806E0A068401BB04202D32C
:1046D0000120BDE8F081384600F003F80028F3D14E
:1046E000F7E770B5044600BF00BF00BF00BF00BFC2
:1046F00000BF00BF00BF00BF00BF00BF00BF00BFC2
:1047000000BF00BF00BF00BF00BF00BF00BF00BFB1
:1047100000BF00BF00BF00BF00BF00BF00BF00BFA1
:1047200000BF00BF00BF1C4E4FF48025F56305207D
:10473000FEF71CF80020FEF719F82070B56300BFE3
:1047400000BF00BF00BF00BF00BF00BF00BF00BF71
:1047500000BF00BF00BF00BF00BF00BF00BF00BF61
:1047600000BF00BF00BF00BF00BF00BF00BF00BF51
:1047700000BF00BF00BF00BF00BF00BF00BF207868
:1047800000F0010070BD00006C000010700000100F
:10479000740000100080004000C009200020704715
:1047A000B04982200860B049212008607846AF49AE
:1047B000086082207047AB4982200860AA49222005
:1047C00008607846A949086082207047A549822080
:1047D0000860A549222008607846A4490860822024
:1047E00070472DE9F041002400BF00BF00BF00BFAB
:1047F00000BF00BF00BF00BF00BF00BF00BF00BFC1
:1048000000BF00BF00BF00BF00BF00BF00BF00BFB0
:1048100000BF00BF00BF00BF00BF00BF00BF00BFA0
:1048200000BF00BF00BF00BF914D4FF08066EE6338
:104830003712EF639F20FDF799FF0020FDF796FFE9
:1048400060F307040020FDF791FF60F30F240020C0
:10485000FDF78CFF60F31744AE63AF6300BF00BF8A
:1048600000BF00BF00BF00BF00BF00BF00BF00BF50
:1048700000BF00BF00BF00BF00BF00BF00BF00BF40
:1048800000BF00BF00BF00BF00BF00BF00BF00BF30
:1048900000BF00BF00BF00BF00BF00BF7549601A66
:1048A0008C421BD00BDCA4F1C204B4F5A11415D0CA
:1048B000B4F5803F12D0B4F5003F0BD10EE06E4945
:1048C000401805D06D4940180AD06D49C84201D141
:1048D000022400E000242046BDE8F0810324FAE72A
:1048E0000424FFF781FBF6E76648007828B16649A3
:1048F00000EBC00051F8200000475A4982200860B0
:10490000594921200860784658490860822070473C
:1049100070B5FFF766FF5B49534D544E514C08701C
:1049200050B1594900EBC00001EB8000806880471E
:10493000000609D5206870BD8220206021202860F3
:1049400078463060822070BD002020602860784664
:104950003060002070BD2DE9F0414A4B424D434E7E
:104960001B78404C5BB192B1474F03EBC30307EB9D
:1049700083031B699847000611D52068ACE78220A5
:10498000206021202860784630608220A4E78620BD
:104990002060092028607846306086209CE700204F
:1049A0002060286078463060002095E72DE9F041CE
:1049B000344B2D4D2D4E1B782A4C5BB192B1324FAA
:1049C00003EBC30307EB83039B699847000611D5EC
:1049D000206881E7822020602220286078463060AD
:1049E000822079E7862020600920286078463060A0
:1049F000862071E700202060286078463060002023
:104A00006AE7F8B51F4C184D184E2778154CDDF89D
:104A100018C087B1BCF1000F15D0CDF800C0DFF889
:104A200068C007EBC7070CEB8707FF69B8470006AC
:104A300011D52068F8BD82202060222028607846A9
:104A400030608220F8BD86202060092028607846EA
:104A500030608620F8BD00202060286078463060F5
:104A60000020F8BD6C0000107000001074000010F1
:104A700000C00920C220180003FBD6FF00FFFEFF84
:104A80000001F8FF180100108C54000070B50646B4
:104A9000FBF7A0FC056806F10B0020F00704B44208
:104AA0009CBF002070BD2B466A68BAB11068A04256
:104AB00010D304F1080188423CBF5068586007D306
:104AC0005168101941601168091B01605860146039
:104AD000101D70BD13465268002AE7D121462846B2
:104AE00000F0C5F80028DED170BD70B50446051F82
:104AF000FBF770FC0068002C14BF446870BD002CEC
:104B000018BFAC423CBF20466468F8D301680A185D
:104B1000AA4218BF456003D12A68054611440160C6
:104B200028684119A1421CBF6C6070BD6168696052
:104B300021680844286070BD032A40F2308010F0DC
:104B4000030C00F0158011F8013BBCF1020F624428
:104B500098BF11F801CB00F8013B38BF11F8013BB9
:104B6000A2F1040298BF00F801CB38BF00F8013B66
:104B700011F0030300F02580083AC0F0088051F8D6
:104B8000043B083A51F804CBA0E80810F5E7121DE1
:104B90005CBF51F8043B40F8043BAFF30080D20700
:104BA00024BF11F8013B11F801CB48BF11F8012BCC
:104BB00024BF00F8013B00F801CB48BF00F8012BEF
:104BC000704710B5203AC0F00B80B1E81850203A79
:104BD000A0E81850B1E81850A0E81850BFF4F5AF9D
:104BE0005FEA027C24BFB1E81850A0E8185044BF27
:104BF00018C918C0BDE810405FEA827C24BF51F894
:104C0000043B40F8043B08BF7047D20728BF31F887
:104C1000023B48BF11F8012B28BF20F8023B48BFD8
:104C200000F8012B70474FF000020429C0F01280F9
:104C300010F0030C00F06080CCF1040CBCF1020F0A
:104C400018BF00F8012BA8BF20F8022BA1EB0C0124
:104C500000F052B85FEAC17C24BF00F8012B00F8D5
:104C6000012B48BF00F8012B70477047704738B5DB
:104C700004460A4600206946AFF30080002808BFBA
:104C800038BD02460099204600F05BF8012038BD8F
:104C90000120FBF7AFBBF8B5AFF30080054600205D
:104CA0000C46102000BF0646A819A0420DD9324676
:104CB00069460020AFF30080070008BFFBF79AFBAE
:104CC0000098A04218BF0546C419FBF783FB056096
:104CD0000746F01D20F0070046192846FBF77EFB2B
:104CE000B44208BFF8BDA21B31463868BDE8F840A1
:104CF00000F027B84FF0000200B5134694469646E0
:104D0000203922BFA0E80C50A0E80C50B1F12001DE
:104D1000BFF4F7AF090728BFA0E80C5048BF0CC08C
:104D20005DF804EB890028BF40F8042B08BF7047EA
:104D300048BF20F8022B11F0804F18BF00F8012B5C
:104D40007047034640688C46002818BF88423CBF25
:104D500003464068F8D318681844884207D00CF11D
:104D6000030020F00700001D411A521A0146081DD9
:104D70000A60FFF7BABE7546FBF738FBAE46050082
:104D80006946534620F00700854618B020B5FBF76A
:104D900015FABDE820404FF000064FF000074FF035
:104DA00000084FF0000B21F00701AC46ACE8C00949
:104DB000ACE8C009ACE8C009ACE8C0098D46704752
:104DC00010B50446AFF300802046BDE81040FBF765
:104DD000C8B9002801D000F029B8704710B50128E3
:104DE00005D0002103A000F027F8012010BD09A183
:104DF000F8E7000053494752544D454D3A204F754E
:104E000074206F662068656170206D656D6F7279C2
:104E1000000000003A2048656170206D656D6F727A
:104E20007920636F7272757074656400014918208F
:104E3000ABBEFEE72600020070B505460C460A2010
:104E400000E06D1C00F011F835B128780028F8D189
:104E500002E0641C00F009F814B120780028F8D1B1
:104E6000BDE870400A20AFF3008008B569468DF8B0
:104E700000000320ABBE08BD00050F0A1B1E141165
:104E800033363C39282D272263666C69787D77722A
:104E900050555F5A4B4E4441C3C6CCC9D8DDD7D21A
:104EA000F0F5FFFAEBEEE4E1A0A5AFAABBBEB4B10A
:104EB00093969C99888D878283868C89989D9792FA
:104EC000B0B5BFBAABAEA4A1E0E5EFEAFBFEF4F1EA
:104ED000D3D6DCD9C8CDC7C240454F4A5B5E5451DA
:104EE00073767C79686D676223262C29383D3732CA
:104EF00010151F1A0B0E040103060C09181D1712BA
:104F000030353F3A2B2E242160656F6A7B7E7471A9
:104F100053565C59484D4742C0C5CFCADBDED4D199
:104F2000F3F6FCF9E8EDE7E2A3A6ACA9B8BDB7B289
:104F300090959F9A8B8E848180858F8A9B9E949179
:104F4000B3B6BCB9A8ADA7A2E3E6ECE9F8FDF7F269
:104F5000D0D5DFDACBCEC4C143464C49585D575259
:104F600070757F7A6B6E646120252F2A3B3E343149
:104F700013161C19080D070200002110422063308F
:104F80008440A550C660E770088129914AA16BB1A1
:104F90008CC1ADD1CEE1EFF1311210027332522249
:104FA000B5529442F772D662399318837BB35AA3F1
:104FB000BDD39CC3FFF3DEE3622443342004011419
:104FC000E664C774A44485546AA54BB52885099541
:104FD000EEE5CFF5ACC58DD55336722611163006E9
:104FE000D776F6669556B4465BB77AA71997388791
:104FF000DFF7FEE79DD7BCC7C448E5588668A778A9
:105000004008611802282338CCC9EDD98EE9AFF9E0
:10501000488969990AA92BB9F55AD44AB77A966A88
:10502000711A500A333A122AFDDBDCCBBFFB9EEB30
:10503000799B588B3BBB1AABA66C877CE44CC55C58
:10504000222C033C600C411CAEED8FFDECCDCDDD80
:105050002AAD0BBD688D499D977EB66ED55EF44E28
:10506000133E322E511E700E9FFFBEEFDDDFFCCFD0
:105070001BBF3AAF599F788F8891A981CAB1EBA124
:105080000CD12DC14EF16FE18010A100C230E320A0
:105090000450254046706760B9839893FBA3DAB348
:1050A0003DC31CD37FE35EF3B1029012F322D232F0
:1050B0003542145277625672EAB5CBA5A895898518
:1050C0006EF54FE52CD50DC5E234C324A014810440
:1050D0006674476424540544DBA7FAB79987B897E8
:1050E0005FE77EF71DC73CD7D326F2369106B01690
:1050F00057667676154634564CD96DC90EF92FE9A8
:10510000C899E9898AB9ABA94458654806782768DF
:10511000C018E1088238A3287DCB5CDB3FEB1EFB87
:10512000F98BD89BBBAB9ABB754A545A376A167A2F
:10513000F10AD01AB32A923A2EFD0FED6CDD4DCD57
:10514000AABD8BADE89DC98D267C076C645C454C7F
:10515000A23C832CE01CC10C1FEF3EFF5DCF7CDF27
:105160009BAFBABFD98FF89F176E367E554E745ECF
:10517000932EB23ED10EF01E005EBCE2613FDD8395
:10518000C29C7E20A3FD1F419DC3217FFCA2401E27
:105190005F01E3BD3E6082DC237D9FC1421CFEA017
:1051A000E1BF5D0380DE3C62BEE0025CDF81633D07
:1051B0007C22C09E1D43A1FF4618FAA427799BC5F7
:1051C00084DA3866E5BB5907DB856739BAE40658E7
:1051D0001947A5FB7826C49A653BD987045AB8E6D7
:1051E000A7F91B45C6987A24F8A6441A99C7257BC7
:1051F0003A6486D85B05E7B98CD2306EEDB3510FB7
:105200004E10F2AC2F7193CD114FADF3702ECC92A6
:10521000D38D6F31B2EC0E50AFF1134DCE90722C96
:105220006D33D18F0C52B0EE326C8ED0530DEFB186
:10523000F0AE4C1291CF2D73CA947628ABF5174976
:105240000856B4EA6937D58B5709EBB536688AD466
:1052500095CB2977F4AA4816E9B7550B88D6346A56
:105260002B7597C94A14F6A8742AC896154BA9F746
:10527000B6E80A54D7896B35EB3C904D53444F53F5
:10528000352E3000020201000110000004F80C006D
:10529000010001000000000000000000000029EFF4
:1052A000BEADDE41544F4C20465072696E7446418B
:1052B00054313220202000000000000000100000C7
:1052C00000200000003000000040000000500000FE
:1052D00000600000007000000080000000900000EE
:1052E00000A0000000B0000000C0000000D00000DE
:1052F00000E0000000F0000000000100008001005C
:105300000000020000800200000003000080030093
:10531000000004000080040000000500008005007B
:105320000000060000800600000007000080070063
:10533000FF0F0000FF1F0000FF2F0000FF3F0000D5
:10534000FF4F0000FF5F0000FF6F0000FF7F0000C5
:10535000FF8F0000FF9F0000FFAF0000FFBF0000B5
:10536000FFCF0000FFDF0000FFEF0000FFFF0000A5
:10537000FF7F0100FFFF0100FF7F0200FFFF02002F
:10538000FF7F0300FFFF0300FF7F0400FFFF040017
:10539000FF7F0500FFFF0500FF7F0600FFFF0600FF
:1053A000FF7F0700FFFF070012011001000000400F
:1053B00051C2031300010420480109022000010129
:1053C00000803209040000020806506207058202CC
:1053D0004000000705020240000000040309041C0D
:1053E00003410054004F004C00200020002000200A
:1053F000002000200020002000200028034600504C
:1054000000720069006E007400200046006C0061AC
:1054100000730068002000200020002000200020F1
:105420000020001A034600690072006D00770061D9
:10543000007200650030003000300030000E034D77
:105440000065006D006F0072007900005D220000B1
:1054500000000000930300000000000000000000B6
:10546000000000000000000000000000000000003C
:10547000000000000000000000000000000000002C
:105480000000000000000000000000009D47000038
:105490009D470000A1470000B7470000A14700005A
:1054A000B7470000B7470000B7470000CD470000EE
:1054B0009D4700009D470000A1470000B74700003E
:1054C000A1470000B7470000B7470000B7470000FA
:1054D000CD4700005B3E0000613E00004B3C0000F9
:1054E0005B3D000091390000C539000079350000AE
:1054F0009B3A0000673E0000932F0000992F0000A8
:10550000952A00005B3D000091390000EF2C00005F
:105510009B420000E32D00009F2F0000AF460000DB
:10552000B54600004B3C00005B3D00009139000097
:105530002B4400009B42000001450000673E000034
:10554000000000000000000000000000000000005B
:10555000000000000000000000000000000000004B
:105560000000000084550000000000101C01000035
:1055700008010000A05600001C0100109C6C0000F7
:105580002401000041544F4C20465072696E74282B
:1055900000000000000000000000D4284B3D000087
:1055A00000000000000000000000000000000000FB
:1055B00000000000000000000000000000000000EB
:1055C00000000000000000000000000000000000DB
:1055D00000000000000000000000000000000000CB
:1055E00000000000000000100000000000000000AB
:1055F00000000000000000000000000000000000AB
:10560000000000000000000000000000000000009A
:10561000000000000000000000000000000000008A
:10562000000000000000000000000000000000007A
:10563000000000000000000000000000000000006A
:10564000000000000000000000000000000000005A
:1056500000000000000000000000000000093D0004
:10566000000000000000000000000000000000003A
:10567000000000000000000000000000000000002A
:10568000000000000000000000000000000000001A
:10569000000000000000000000000000000000000A
:1056A000FC5F9BEFC957B1CAE0D1298055BD9E3C34
:1056B0003DBA0F02C0F67BC9C8196F82DAD7518E86
:1056C00098834663F2513AE8BDB1987E29F51B4DA7
:1056D000A50D80597AF171F83FC0D7C9AEF985A7F9
:1056E00087ECDC7CEFE6CB4E95CCB7C3278CB46B54
:1056F000973D94C2EB37A0392CAF27C1DBF70FA33E
:1057000044C0189AF65DB040D0EEC9309FA76692AB
:1057100045DD3B2341D5D135318894C619B3E273B9
:10572000C324D9A7870E696CB21970813C38520422
:10573000BE4203FA3AE25FFC593648C7C351253EE0
:10574000C535727AE7FDD40F6644100BE8E4C3F266
:105750001162E46CA82A4B2FFFD519ADAEC6A17F0C
:10576000D4B8E8BBB729A7D728E5C64033F7AE3B86
:10577000ADAF2AD4747E6DAB661342BA09AFFA623C
:10578000A9FBF56DC3D260A6E2B900CBAE25819D21
:10579000FFEF41545DD30B40EBA2FFB96AE14E87A6
:1057A00014E7C0F957E3855F78DD1084FD093DC932
:1057B000845BCB3F9F4ED84084DF1708E2DB057B3C
:1057C000AAF311E472C4035241428D9A3715CE7484
:1057D000DFBBEBFEEAC2AA98BE28550DFEBF24A28D
:1057E000FF7E33AC14132F5558F046FA8B9C6D9BFB
:1057F0000F888D891EA675893D4FC9E93EED536519
:105800004DD88384FE43BC4D2B8EB83518D0130C75
:105810006B7CA6E2E4CF4FE616A76D93D5022FD797
:10582000C5D02921F1D66A14AC77794319679776E8
:10583000DD433B7124876419BC664B8BEBE0137F1F
:10584000FA03C03C47760982EF283B930C01AFB9BD
:105850002E7D63C88F4239AE1F1915EEDDF510F8A5
:10586000AFC01D83C42199AF30982955A5C29C5C57
:105870000E734D3EC3C556170E95F0B7418B176F8B
:10588000A76E8386A77453FC81192025DAAF48667A
:10589000EC39993A16CCE63C7B4883D7557D994341
:1058A0006DD8292A8A19BDE1D54D4061907DC3C7C5
:1058B000F310B16613A5DF94B357E90CA3C0EB2234
:1058C000396B8B8938EA70AB47A419A7273D6C5C0C
:1058D000B416BF5868EE243830AAA64BCBB60422C3
:1058E000EE966D15ECC18C3D54A408FF673F035D37
:1058F00003554F1D738468BCE7D098810221DA32CA
:10590000996FAF0D6DF60ACD16570D913F3873495B
:10591000F95E540C70C02CFF3518C3DAF84994DBDB
:105920003FA6BFEEFD585360F51B5AEF28435D6458
:10593000171CAC70218DC8D7F7F5533953D4AC89F7
:10594000BEE5FBED749B7D4EBD8DEB5D707DCFBCE8
:10595000FA3511742BB8260EBAEA1C565249A52402
:105960000C66138CC26E6FA4FBA43BD1B4869EEC74
:105970004AF0DB4D0997C643DC0D9C8BED90160475
:105980006AC19452FE606B74209E111E203E7E7A86
:105990004EEAA241F93F08AAD018C690092498B34C
:1059A000BB633D4DCDC140788301FBBCBF832DEC73
:1059B000E59F33948D642F03DBB933A8B76ED26EA5
:1059C00050B51458FC045169ED98F9BD29D246C66A
:1059D000222E84D28541FAAE287EE4A3022A9D8D30
:1059E00075176BFACA5DE0A32FF6332D0B68F0A78D
:1059F00042397D119A5D7D92662343534C39FC09EF
:105A000070286A1C6ABB1AF6BD88F157C60EC15AC7
:105A100030F393B527266AF6A925ED3EC8043AD49B
:105A20005ED215474DDBC88223B367A2FA87C263F3
:105A30000E5646864850F8C84DF124DA82CA79A23B
:105A400080F7337629D34F497B64332B18EF282C0A
:105A5000A7345B88FC20C77EA22C9513D256C75C66
:105A60002FFBF568B2E183FF875C40E50258BCE696
:105A7000217EFAE278DA186495BFCAFF47857C0A6E
:105A800020842A097B71E0E5B182BD980D3DAEF519
:105A90005BBB0DE1F58A5FB40772488E74D42DBFED
:105AA000D4D85E0EC24DF4CC9311B5EFD8D75CF6C6
:105AB000634F752055C285BA7F8ECBC5127A43D10C
:105AC00033686D27260874675931316CEC3E382CE9
:105AD0001013B20D4B6CB1D2DDFD966829D791CA77
:105AE0007CB9220C329F72832E6429C7215C9F8669
:105AF0002405E6CFCAE9E602F44DC75B695E4EEFC6
:105B0000C056CBA7C5B26271038F90BBEFAB5709EC
:105B1000B2D3A2AD4C906ACCE059857C0FE3BC1B9C
:105B2000CB5B15EA3D209637EE35E9A2777215403A
:105B30008B2F819115C076DE05240F825772A477D2
:105B400039C874DA9A5DFAE4F855B8F723F1CA83D4
:105B5000724D242430BA2C02DBFB1E722F1C5379A9
:105B6000B6B84006DC93AA19AB8E4A93C7F74A141D
:105B700008CDCEA65E1FA97D6DA06386903B471F12
:105B800005C45F1C4CCDC92C26CDDC078CF93F2801
:105B900073170358C28E8A99C330DA55F7F5AB7D77
:105BA000BC7D297BE010FA59FA3A99144CCF983C05
:105BB000EFE34988B8403E2E354FDDFB44001B32F1
:105BC0007EF4892FC28205482B1CAFB5FA3BF53A0B
:105BD000754EE7124237282ABDD4B2DA1B741C86F0
:105BE000C8CB86C14A82280CEC6EC0EFF91844700D
:105BF0005438669206C523B8E58B52B992D2CA0FC3
:105C000036C5162566FDA4DA991ED6A527D1FA0950
:105C100051528B53193F0FF7A2B7557E2195D88764
:105C200026AE633D8E3E19DA6C6B3FB3B61F092674
:105C30005027DE5A394AB986A454F368A25D123B54
:105C40001D6B133666CF2B704558B86A32373188D2
:105C50000B5C2616393CADF0C91FC01AD15F9ECA35
:105C6000E5E371D7048F458F0F57EB8134A13A4498
:105C7000E7759BFE6D634728320065371161B024DC
:105C800058DAC17E246CBAFEF436C8ED952A1F3668
:105C90009DB0E778A66EA2D5712A8466AD123598BC
:105CA000A49C060987D190B4BDCE92583A6A3A476F
:105CB0001E33A7BA0EA47339A6A93464FAF2E78991
:105CC00071EE116A04EE212F7BBCFB3C8031FC9706
:105CD0006BD6C61FFBC9F541774D57B8CCD7E20B41
:105CE0004E6FDA9BF924393550EDA07753E0C98720
:105CF00089764898BE101D4A7885C000EFAFE57FD1
:105D0000E5DF31BB039D692D405B9380B7ECC84351
:105D1000ADF72EC88F47774752D890F2AAC9CDE881
:105D20000102129DE6FA3F85B78FDA77CFF9A846D0
:105D300066CBF69B0C120B6F5DDF7E0DA67BAE3043
:105D4000AF5F57B629BC3B470D3B3500C8028F23D8
:105D50005C6D3E4D00BA3FAF3C238E71EB497C3801
:105D600052C983786D984F10E3D6B5E2C0F5064E60
:105D700050D2D3399307AFF234FF3B3A94D3B0CE2D
:105D80000BE1CABEF3FDF78495C66494D749632D31
:105D9000D0849DAAE63373AC215305F9DFF25D9000
:105DA000FCFFD131E83657A483A5B6A44CAB955F70
:105DB0009BCD4786F559EE26481A293D775A73122E
:105DC000926C2F4FF9DFD11BEB28A0D37512C5DFE2
:105DD0004BAEC57156723B23C1AAEE5211E00713B8
:105DE00073EDA5F7F3A8E9C6F4D500E11BA8EEF220
:105DF0009A391451291CBE858B2CBBAF572B5A7571
:105E00006B4B3C2309B0376E9D33428E132DC182FC
:105E100032FA3C67BFEAE382273C326A569865EE65
:105E200053EEC8E1A9E811080A4BC86D18FCC35C21
:105E30000EEAFA318F6A67629E0D3DF1871867E6B8
:105E4000655D62806BD208CB6CD010EF224BE118FD
:105E500070A6023690EF01DB90322E44DD5115938F
:105E600029D4BFC6AFD007AC8FBA3938BD1D9C321C
:105E7000333D00C3F07C2A3FF4362F3935AC1F2A5E
:105E80006881678A334A1424F586166465A05055E4
:105E9000753139F5CFA2350B23E80FB1EDD3EB7D8A
:105EA00034B33F28D157078E23E92813E451FAFA77
:105EB0005D0D738F499D6EEE956C9F7662D383ACBA
:105EC000C2DE24F91D483732EE9D6EE6652A9979C7
:105ED000314ABF95303AB3EAF105C685C3722D0445
:105EE0002FBFF66DE9D6CAF5F717F7E7407201AA9A
:105EF000F868DFD8DF9FCBEFFE9C41F3E4023D560C
:105F000003C176E0C362E4806B7EE801D2B68050C4
:105F100091A2C8A781EA6FF52BB734D8A8E852A898
:105F2000E292183B919F5071D1C9F696A4916F0BE4
:105F3000CA405B160DC80290CA7BC3884E95DDC966
:105F4000D345C411F769CABAA1464B0716821FA2EE
:105F50002DBC2B6564D573F17AD54522736F9CA84F
:105F6000BA17A6D8C2AC35D4F611B2B48850F69C94
:105F700095C98CE1BFEA152CA12D34C44699804106
:105F80006EC4EB1A3C7FBB7E173BB7BFA3C0E7D400
:105F900019FC8B15993C95464ABED2038ADAF83C27
:105FA00030FA73631B879087074AC0A0B2EA87CC98
:105FB0006CD2DB287CE8F2C9FC7E1C2A691D1EF12C
:105FC000E2BEFCEA930BAFE02163E3F7537C72AFD0
:105FD0002354B0F1F29CEB56F1DA69E6AC91DCE6C1
:105FE00035BF25ADA9632D19700F96D45961367B45
:105FF0005B68BB21CBC1297B86ABD40FFB97898221
:00000001FF
